:020000040000FA
:020000007C2D55
:080008008801803123309500CE
:10001000A10A063021020318A1012014A20F1328FF
:10002000A30F1328A0143D08003E031932282E1CEC
:1000300030288801880ADB308D0088018D010D157C
:10004000452301304F2300001E30A4000D1107305E
:100050004F230D1506304F23A40B26280D115328CE
:10006000452334283A2333231430A500FD01FC0135
:10007000D921DF21ED213E23210803195920013028
:10008000210203199920023021020319D9200330DB
:1000900021020319192104302102031959210530C5
:1000A0002102031999218E018C018D018E010B1102
:1000B0000900B830840015080002031C7C17B93011
:1000C000840015080002031CFC167C16BA3084005C
:1000D00015080002031CFC15BB3084001508000243
:1000E000031C7C15A330840015080002031CFD16B8
:1000F000A230840015080002031C7D16FD15A130F6
:10010000840015080002031C7D15A030840015082A
:100110000002031CFD148801880A7D088C007C08FD
:100120008D00880180308D0001308C00A50B59288E
:100130000800BC30840015080002031CFC17BD3009
:10014000840015080002031CFC16BE30840015084C
:100150000002031C7C16FC15BF3084001508000249
:10016000031C7C15A730840015080002031CFD1633
:100170007D16A630840015080002031CFD15A5306D
:10018000840015080002031C7D15A43084001508A6
:100190000002031C7D148801880A7D088C007C08FD
:1001A0008D00880140308D0002308C00A50B99280D
:1001B0000800C030840015080002031CFC17C13081
:1001C000840015080002031C7C17C2308400150847
:1001D0000002031C7C16C330840015080002031CB7
:1001E000FC157C15FD16AB30840015080002031CBD
:1001F0007D16AA30840015080002031CFD15A930E5
:10020000840015080002031CFD14A83084001508A2
:100210000002031C7D148801880A7D088C007C087C
:100220008D00880120308D0004308C00A50BD9286A
:100230000800FC17C430840015080002031C7C175A
:10024000C530840015080002031CFC16C63084006B
:1002500015080002031CFC15C730840015080002B5
:10026000031C7C15AF30840015080002031CFD162A
:10027000AE30840015080002031C7D16AD308400EA
:1002800015080002031C7D15AC308400150800021F
:10029000031CFD147D148801880A7D088C007C08ED
:1002A0008D00880110308D0008308C00A50B1929B5
:1002B0000800C830840015080002031CFC177C17D6
:1002C000C930840015080002031CFC16CA308400E3
:1002D00015080002031C7C16CB30840015080002B0
:1002E000031C7C15B330840015080002031CFD16A6
:1002F000B230840015080002031CFD15B1308400E3
:1003000015080002031C7D15FD14B030840015088B
:100310000002031C7D148801880A7D088C007C087B
:100320008D00880108308D0010308C00A50B5929F4
:100330000800CC30840015080002031CFC17CD30E7
:10034000840015080002031C7C17FC16CE308400C4
:1003500015080002031C7C16CF308400150800022B
:10036000031CFC15B730840015080002031C7D1621
:10037000B630840015080002031CFD157D15B5304C
:10038000840015080002031CFD14B4308400150815
:100390000002031C7D148801880A7D088C007C08FB
:1003A0008D00880104308D0020308C00A50B992928
:1003B00008000310260DAF00E621B200080003106C
:1003C000260D013EAF00E621B300080001308A008F
:1003D0002F08F13E03188A0A820032088A00330887
:1003E00082000234313402343C3402344434023466
:1003F0004C340234543402345C34023464340234F5
:10040000703402347434023480340234843402345C
:100410009034023494340234A0340234A4340234CC
:10042000B0340234B4340234C0340234C43402343C
:10043000D0340234D4340234E0340234E4340234AC
:10044000F0340234F4340334003403340434033419
:100450001034033414340334203403342434033488
:1004600030342D103030B1002818392A0630A6005B
:10047000322B0130A600322B2818412A0030A6006A
:10048000322B0230A600322B2818492A0030A60051
:10049000322B0330A600322B2818512A0430A60034
:1004A000322B0330A600322B2818592A0030A60020
:1004B000322B0530A600322B2818612A0730A600FF
:1004C000322B0030A600322B28186E2A003031075C
:1004D00003196C2AB10B322B2D14322BA601322BAF
:1004E0002808AC00A60A322B2C082806031D7A2AFD
:1004F000A601322B28182B10281C2B14A60A322BED
:100500002808AC00A60A322B2C082806031D8A2ACC
:10051000A601322B28182A12281C2A16A60A322BCA
:100520002808AC00A60A322B2C082806031D9A2A9C
:10053000A601322B2818AA11281CAA15A60A322BAC
:100540002808AC00A60A322B2C082806031DAA2A6C
:10055000A601322B28182A11281C2A15A60A322B8C
:100560002808AC00A60A322B2C082806031DBA2A3C
:10057000A601322B2818AA10281CAA14A60A322B6E
:100580002808AC00A60A322B2C082806031DCA2A0C
:10059000A601322B28182A10281C2A14A60A322B4E
:1005A0002808AC00A60A322B2C082806031DDA2ADC
:1005B000A601322B2818A912281CA916A60A322B2C
:1005C0002808AC00A60A322B2C082806031DEA2AAC
:1005D000A601322B28182912281C2916A60A322B0C
:1005E0002808AC00A60A322B2C082806031DFA2A7C
:1005F000A601322B2818A911281CA915A60A322BEE
:100600002808AC00A60A322B2C082806031D0A2B4A
:10061000A601322B28182911281C2915A60A322BCD
:100620002808AC00A60A322B2C082806031D1A2B1A
:10063000A601322B2818A910281CA914A60A322BAF
:100640002808AC00A60A322B2C082806031D2A2BEA
:10065000A601322B28182910281C2914A60A322B8F
:10066000A601301408002D10AD108E1E2D148E1F03
:10067000AD14080028100E1B2814080027082602B5
:10068000031C442B2608A70008002E10BD030310EE
:10069000BC0CBB0CBA0CB90C03182E140800B40027
:1006A000B40B502B0800BA01BB01BC01A030B9004B
:1006B000B709371C3A143718BA14351E3A15351ACB
:1006C000BA15B51D3A16B519BA16351D3A173519AA
:1006D000BA17B51C3B14B518BB14351C3B1535189F
:1006E000BB15B61E3B16B61ABB16361E3B17361A7E
:1006F000BB17B61D3C14B619BC14361D3C15361973
:10070000BC15B61C3C16B618BC16361C3C17361861
:10071000BC172130BD000800BE01BF010830C00079
:100720000310C20CBF0DBE0DC10CBF0DBE0DC00B22
:10073000902B0800C300C4010830C5000310C30C8F
:10074000C40DC50B9E2B44080800C6000000C60B54
:10075000A62B0800CD0A4D080F3C0319CD014D080A
:10076000B800FB01FA010800CD034D08013E031D4E
:10077000BC2B0E30CD00B800FB01FA01080029089F
:10078000CD00B800F13E031CC92B0E30CD024D0840
:10079000C22BFB01FA010800C7002010201CCE2B41
:1007A000C70BCD2B08004D0A9A23CF00D001D101F1
:1007B000D201D301D40170305718D000FF30C824C3
:1007C000CF01D001D1010130C82408000530C80094
:1007D000CB30C90003104D0DFB008B13BE258B17CA
:1007E000CA0003144D0DFB008B13BE258B17C900E7
:1007F0004A08C800080021304802031D032C49089C
:100800007B072C24152C8B130A08CB0048087A0789
:10081000DB00031049087B07DC000318DB0AC52551
:10082000CC004B088A004C088B17FB0F182CFA0AD7
:100830000800230095181A2C8B13151523007B082C
:10084000910079089300230055309600AA30960055
:1008500095148B17880108008B13230095182E2CF4
:10086000151123009100230095131514230013087C
:1008700088018B17080000302C24D70008003B2487
:10088000571C442C5710452C57140030FB005708B8
:10089000F9001924D323D3230800E623FB01FA012E
:1008A000FB23CE00CE13FB23D600D60AFB23D800B1
:1008B000301C762C07302A02031D612CBF23B001A7
:1008C0004D2CAA08031D762C203029020319AA23D7
:1008D000213029020319B423003029020319CD0164
:1008E0000C30290203193F24B0014D2C2D080319A7
:1008F0008C2CD323D32303302D0203193F242D182E
:10090000842CAD18882C4D2CAA23D323D3237B2CE5
:10091000B423D323D3237B2C17304E028431031905
:10092000B52484311B304E028831031900288431EC
:100930003D08003E031DA82CA01CA82CA010571C8D
:10094000A32CAA234D2C0730B5003808B60053233A
:10095000D80B582C4D2C590D590D591A013AD91A4A
:10096000013AD919013AD9000800FB23CF00FB2333
:10097000D000FB23D100FB23D200FB23D300FB23B9
:10098000D4003030DA005608C824DA0BC32C080033
:10099000D500AE3084008001D21B8009B3308400C2
:1009A0008001521B8009AF3084008001D21A800977
:1009B000AB3084008001521A8009AA308400800183
:1009C000D2198009A2308400800152198009A33015
:1009D00084008001D2188009A73084008001521859
:1009E0008009A63084008001D31B8009A5308400D3
:1009F0008001531B8009A13084008001D31A800933
:100A0000A03084008001531A8009CC30840080011A
:100A1000CF1B8009C830840080014F1B8009C9307A
:100A200084008001CF1A8009CA30840080014F1AE7
:100A30008009CE3084008001CF198009CF30840036
:100A400080014F198009C13084008001CF188009CE
:100A5000BC30840080014F188009C03084008001C0
:100A6000D01B8009C43084008001501B8009C53030
:100A700084008001D01A8009CD3084008001501A92
:100A800080095508CC23080002302602031C03010C
:100A9000CF000030D0000130C8242D080319602D8C
:100AA000A701A6013D08003E031D4D2D2D08D000D5
:100AB000CF010130C824B5010C30B60053234D2DB1
:100AC000301C442DB001F030CF00D0017F30C8245D
:100AD000CF01D0013F30C824F030CF00D0017F30AB
:100AE000C8242908CF002A08D000FF30C824FF30CE
:100AF000C824A701A601442D8C019501CD01BD019B
:100B0000AB01AA01A901AC01A601A701B001A10195
:100B1000A201A301AD0121007230990023008C01D4
:100B200022008C0122008D0123008D0121008230E2
:100B300095002100E0308E002000AD011D30D9006D
:100B40008B168B17FF30CF00D000D100FF30C824A8
:100B5000FF30C824CF01D001D101FF30C824FF30BD
:100B6000C824FF30C8243B242D08D000FF30C824FF
:100B7000FF30C8242D1C4D2C3F24442D48088A00EA
:100B80007B08490703188A0A82000A08CB005B0821
:100B90008A005C0882000834B2340834FD34093419
:100BA000123409345D34093478340934DB340934BF
:100BB000F0340A3423340A3438340A344D340A34D5
:100BC00074340B342B340B347C340B34CD340B3471
:020BD000F434FB
:101000005608D5008331FB23CF00FB23D000FB2300
:10101000D100FB23D200FB23D300FB23D400883173
:101020006430BF00AE308400D21BAA20D21FAE2095
:10103000B3308400521BAA20521FAE20AF30840070
:10104000D21AAA20D21EAE20AB308400521AAA2097
:10105000521EAE20AA308400D219AA20D21DAE2082
:10106000A23084005219AA20521DAE20A330840061
:10107000D218AA20D21CAE20A73084005218AA2071
:10108000521CAE20A6308400D31BAA20D31FAE2052
:10109000A5308400531BAA20531FAE20A13084002A
:1010A000D31AAA20D31EAE20A0308400531AAA203F
:1010B000531EAE20CC308400CF1BAA20CF1FAE2001
:1010C000C83084004F1BAA204F1FAE20C9308400B7
:1010D000CF1AAA20CF1EAE20CA3084004F1AAA20F1
:1010E0004F1EAE20CE308400CF19AA20CF1DAE20D7
:1010F000CF3084004F19AA204F1DAE20C13084008C
:10110000CF18AA20CF1CAE20BC3084004F18AA20D4
:101110004F1CAE20C0308400D01BAA20D01FAE20B0
:10112000C4308400501BAA20501FAE20C53084005C
:10113000D01AAA20D01EAE20CD308400501AAA208A
:10114000501EAE2055088331CC238831BF0B1228A6
:101150008431982C800A0319800908008008031D37
:1011600080030800173410340C3480340034003409
:1011700080340034003440340034003440340034CF
:10118000003420340034003420340034003410346F
:101190000034003410340034003408340034003497
:1011A000083400340034043400340034043400348F
:1011B000003402340034003402340034003401348A
:1011C00000340034013400340034003480340034FE
:1011D000003480340034003440340034003440346F
:1011E000003400342034003400342034003400341F
:1011F0001034003400341034003417341034033405
:10120000FF34FF34FF34FF34FF34FF34FF34F03455
:101210000034FF34F034003400340F34FF34003431
:101220000F34FF34173403340C348034103400345A
:1012300080341034003440342034003440342034BE
:10124000003420344034003420344034003410342E
:1012500080340034103480340034093400340034D5
:1012600009340034003406340034003406340034C9
:10127000003480341034003480341034003440346E
:1012800020340034403420340034203440340034DE
:10129000203440340034103480340034103480342E
:1012A0000034093400340034093400340034063486
:1012B000003400340634003400341734103404345D
:1012C000FC340F34C03400340034003400340034B3
:1012D0000034FC340F34C0340334F0343F34003471
:1012E000003400340034003400340334F0343F342C
:1012F0001B3404341034FF34FF34FF34FF34FF3424
:10130000FF34FF34FF34FF34FF34FF34FF34FF3445
:10131000FF34FF34FF34FF34FF34FF34FF34FF3435
:10132000FF34FF34FF340034003400340034003420
:10133000003400340034003400340034003400340D
:1013400000340034003400340034003400340034FD
:10135000003400340034FF34F0340034FF34F0340F
:101360000034FF34F0340034FF34F0340034FF3400
:10137000F0340034FF34F0340034FF34F0340034FF
:10138000FF34F034003400340034003400340034CE
:1013900000340034003400340034003400340034AD
:1013A000003400340034003400340034003400349D
:1013B000003400340034173403340334DB346D3428
:1013C000B634DB346D34B6346D34B634DB346D345E
:1013D000B634DB34B634DB346D34B634DB346D34E0
:1013E000173402340834803410340034803410341C
:1013F0000034403420340034403420340034A034ED
:1014000050340034A034503400345034A03400340C
:101410005034A0340034293440340034293440346A
:1014200000341634803400341634803400340934E7
:1014300000340034093400340034063400340034FD
:10144000063400340034173403340334DB3460349E
:101450000034DB34603400346D34B03400346D3427
:10146000B0340034B634D03400346D34B034003489
:10147000173403340334923440340034923440340B
:1014800000344934203400344934203400342434C6
:101490009034003424349034003417340334063448
:1014A000C33401348634C334013486346134803427
:1014B000C33461348034C3343034C834613430349C
:1014C000C834613418346C34303418346C343034EB
:1014D0000C34363418340C3436341834863413341F
:1014E0000C34863413340C341B3404341E348034EE
:1014F00000340134003400340034C0340034033488
:10150000003400340034E034003407340034003454
:101510000034F03400340F340034003400347834B4
:1015200000341E340034003400343C3400343C3485
:101530000034003400341E34003478340034003475
:1015400000340F340034F0340034003400340734F5
:101550008134E0340034003400340334C334C03404
:101560000034003400340134E73480340034003473
:1015700000340034FF3400340034003400340034CC
:101580007E34003400340034003400343C34003401
:101590000034003400340034183400340034003493
:1015A000003400340034003480340034013400341A
:1015B00000340034C03400340334003400340034C8
:1015C000E03400340734003400340034F0340034A4
:1015D0000F34003400340034783400341E340034C6
:1015E000003400343C3400343C34003400340034E3
:1015F0001E34003478340034003400340F340034A6
:10160000F03400340034003407348134E0340034E2
:10161000003400340334C334C034013400340034A3
:101620000134E73480340034003400340034FF34B3
:10163000003400340034003400347E34003400348C
:101640000034003400343C340034003400340034BE
:101650000034183400341B3404340D348034103416
:101660000034803410340034C03430340034C0349A
:1016700030340034E03470340034E03470340034FA
:10168000F034F0340034F034F03400347934E034A1
:1016900000347934E03400343F34C03400343D3415
:1016A000C03400341F34803400341F34803400349C
:1016B0000F34003400340F34003400340634003466
:1016C0000034063400340034003400340034003474
:1016D000003400340034003400340034003400346A
:1016E000003400340034003400340034003400345A
:1016F00000340034003400341B3404340D34063418
:10170000003400340634003400340F340034003424
:101710000F34003400341F34803400341F348034DC
:1017200000343F34C03400343D34C03400347934A4
:10173000E03400347934E0340034F034F0340034F0
:10174000F034F0340034E03470340034E034703479
:101750000034C03430340034C03430340034803489
:101760001034003480341034003400340034003439
:1017700000340034003400340034003400340034C9
:1017800000340034003400340034003400340034B9
:101790000034003400340034003417340334063489
:1017A0008034103400348034103400342034403419
:1017B0000034203440340034093400340034093417
:1017C00000340034403420340034403420340034B9
:1017D0001034803400341034803400340634003443
:1017E0000034063400340034173401342134C0345A
:1017F00030340034C0343034003400340034003429
:10180000003400340034C03430340034C034303458
:101810000034003400340034003400340034003428
:101820000C34033400340C340334003400340034FA
:1018300000340034003400340C34033400340C34ED
:1018400003340034003400340034003400340034F5
:1018500000340034003400340034003400340034E8
:1018600000340034003400340034003400340034D8
:1018700000343034C03400343034C03400340034E8
:10188000003400340034003400343034C0340034C8
:101890003034C034003400340034003400340034B8
:1018A0000034003403340C34003403340C3400347A
:1018B00000340034003400340034003403340C3479
:1018C000003403340C340034003400340034003469
:1018D0000034003400340034003400340034003468
:1018E0000034003400340034003400340034003458
:1018F0000034003400340F34003400340F3400342A
:1019000000340034003400340034003400340F3428
:10191000003400340F340034003400340034003418
:1019200000340034003400340034F0340034003427
:10193000F034003400340034003400340034003417
:101940000034F03400340034F03400340034003417
:1019500000340034003400340034003400340034E7
:1019600000340034003400340034003400340034D7
:0A1970000034003400340034003469
:020000040001F9
:02000E0084E983
:02001000FFFEF1
:02E00000FF34EB
:00000001FF
